:1000000051C08DC06AC069C068C067C066C065C0A5
:1000100064C063C062C061C060C05FC05EC05DC0DC
:100020005CC05BC05AC059C058C057C056C055C00C
:1000300054C053C000CDD914F13C28E5A16C78B56B
:10004000509D89441A03540069006C006C00200024
:100050004800610072006200610075006D001A03C3
:100060006900320063002D00740069006E007900A1
:100070002D0075007300620012011001FF000008DE
:10008000030431C605020102000109021200010148
:100090000080050904000000FF00000004030904BB
:1000A0000100FF8E11241FBECFEFD4E0DEBFCDBF15
:1000B00011E0A0E0B1E0EEE3F9E002C005900D929E
:1000C000A630B107D9F711E0A6E0B1E001C01D925A
:1000D000A633B107E1F7EDD230C492CFDC019FEF38
:1000E0008FEF660FB9F044E3F0E0229560FF2D91A9
:1000F000E82FE227EF70929582958F70392F307F2D
:10010000832B9F70E40F35919327317093278327BA
:100110006A9559F7809590958D939D9308950F93C7
:100120001F932F93DF93CF930FB70F934A99FECF6F
:100130004A990BC04A9909C04A9907C04A9905C013
:100140004A9903C001E00CBBA8C0C0911E01DD2785
:10015000C15EDE4F0BE014E124E04A9BE9CF3F9300
:100160004F936F9369B130E803C069B1432B499352
:10017000442764712627215029B12471A9F13795AC
:100180003C3FA0F56227615069B1647137953C3FEF
:1001900098F526272150379529B124713C3F90F5D9
:1001A0006227615037953C3F69B16471A0F52627FD
:1001B000215037953C3FC8F529B124716227615021
:1001C00037953C3FB0F50A9569B17AF064712627FE
:1001D000215037953C3F88F529B124716227615041
:1001E00037953C3F10F22DC031C048C0612729B17E
:1001F00024713F774160C6CF3F77426069B1647137
:100200002127C7CF3F774460612729B12471622736
:1002100061503795C8CF3F7748602127316069B179
:100220006471262721503795C6CF3F7740616127FB
:10023000C1CF3F7740622127C4CF3F774064612719
:10024000C9CF3F774068212700C08FCF31E03CBB4A
:100250000B500195033090F0C01B2881233C91F195
:100260002B3481F119811F7740913501141731F436
:100270002936D9F02D3249F0213E39F044274093F8
:1002800006016F914F913F9108C0209306016F9135
:100290004F913F910CB300FD49CF0F910FBFCF910C
:1002A000DF912F911F910F9118950091100100235C
:1002B000F1F040911D014423D1F440931001C1E1BC
:1002C000D1E018C0209106012223C1F240911D0106
:1002D000442369F400931D0120931C0100911E0129
:1002E0004BE0401B40931E01C0E0D1E002C0C1E0E2
:1002F000D1E001E02BB12B7E20611AB114612BB942
:100300001AB914E130E830FF21272BB9379547950A
:100310004C3FC0F530FF212737952BB947954C3F0F
:10032000A8F530FF2127379500002BB947954C3FA2
:1003300078F530FF2127379500002BB947954C3FC2
:1003400048F530FF212769912BB9379547954C3FE8
:1003500018F530FF212737952BB947954C3F00F50D
:1003600030FF2127379547952BB94C3FD8F430FF04
:1003700021273795362F47952BB94C3FA8F40A957E
:1003800012F614C0212744272BB9C2CF2127C5CF8D
:100390002127CBCF2127D1CF212744272BB9D7CF56
:1003A0002127DACF2127DFCF2127E5CF2B7E2BB9DD
:1003B0006F914F913F9101E00CBBDF91CF911AB14A
:1003C000022F20612BB91B7EDFBFDF912F91000030
:1003D0001AB90BB91F910F911895E9E6F0E08081E9
:1003E00083608083E89A789408951F93CF93DF9376
:1003F00060911D01662309F477C080911E01CCE055
:10040000D0E0C81BD109C15EDE4F81E080930701B7
:1004100080911C018D3209F059C01E818F8181119C
:100420001FEF8881807609F041C08981882321F4FB
:100430001882198292E042C0853021F48A8180932B
:100440000B01BAC0863039F582E0809307018B81B9
:10045000813021F492E1C8E7D0E030C0823021F44D
:1004600092E1CAE8D0E02AC0833009F0A5C08A81B1
:10047000882321F494E0CCE9D0E020C0813021F43D
:100480009AE1C4E4D0E01AC0823009F095C09AE144
:10049000CEE5D0E013C0883019F481E0888304C031
:1004A0008A3009F089C0188291E008C0CE01AFD12E
:1004B000982F8F3F19F483E080930701191708F0F4
:1004C000192FD0930A01C093090105C0635011F0A0
:1004D000CE0114D110E01093080183EC8093110138
:1004E0001092100110921D0180911001882309F0D3
:1004F00053C020910701222309F44AC080911101C1
:1005000098E889278093110110910801193010F0A3
:1005100018E002C0112379F1233031F482E191E037
:10052000612F2AD1182F22C03091090140910A0170
:10053000213061F4832F942FFC01A2E1B1E081917D
:100540008D938E2F831B8117D0F30CC0832F942F94
:10055000FC01A2E1B1E0849131968D938E2F831B33
:100560008117C8F3F0930A01E09309018091080113
:10057000811B8093080182E191E0612FAFDD1D5F57
:10058000109310011350183038F41092070104C072
:1005900080910B01809335018AE002C0815019F0EF
:1005A0004C9BFCCF0BC0F8941092100110921D01CF
:1005B00010920B01789402C090E082CFDF91CF912E
:1005C0001F910895882319F03C98449A08953C9A05
:1005D00044980895E0910401F09105013197F1F7F5
:1005E000882329F03D98459A359BFECF02C03D9A5D
:1005F000459880910201909103010197F1F70895C8
:1006000081E0E8DF80E0E6DF089580E0DBDF81E085
:10061000E1DF81E0D7DF08950F931F93CF93DF933E
:10062000C7E0D0E0082F10E0C8010C2E02C095955D
:1006300087950A94E2F780FF02C081E001C080E064
:10064000C1DFDEDF21978FEFCF3FD80769F781E069
:10065000B9DF81E0BFDF16B180E0BCDF12951F700B
:100660001095812F8170DF91CF911F910F91089587
:10067000FF920F931F93F82E81E0A4DF80E0AADFA2
:1006800017E000E081E0A6DF000F3499016080E010
:10069000A1DF1150B8F7FF2011F081E001C080E028
:1006A00091DFAEDF81E08EDF802F1F910F91FF90F1
:1006B00008952EE088E190E00FB6F894A895809315
:1006C00060000FBE209360003C98449A3D98459A84
:1006D00010920E0110920D018BB18B7E8BB98AB1F5
:1006E00084618AB980E49CE90197F1F78AB18B7E35
:1006F0008AB973DE7894A89578DEFDCFEF92FF92E9
:100700000F931F93CF93DF93E82E292FF62E80911E
:100710000C01813021F500910D0110910E01862F01
:1007200090E00817190708F4F02E8E2D922F9C01E7
:10073000E90102C0899170DF9E012E192F15D0F3B7
:10074000A8014F19510950930E0140930D0180915A
:100750000F0181FF0AC0452B41F457DF06C08E2DE3
:1007600060E070E04F2D50E0E1D0DF91CF911F911C
:100770000F91FF90EF900895CF92DF92EF92FF924A
:100780000F931F93CF93DF93C82E292FD62E8091DE
:100790000C01813061F5E0900D01F0900E01862F83
:1007A00090E0E816F90608F4DE2C8C2D922F9C01BF
:1007B0008901E70108C080E0209709F481E058DF53
:1007C000F80181938F012197802F8C198D1598F353
:1007D00097012D19310930930E0120930D0180915D
:1007E0000F0181FF0AC0232B41F40FDF06C08C2DBF
:1007F00060E070E04D2D50E099D08D2DDF91CF91CC
:100800001F910F91FF90EF90DF90CF9008951F936D
:10081000CF93DF93EC0189818230E9F0833030F4AB
:10082000882359F0813009F073C00DC0833009F47A
:100830006AC0883008F06CC030C08A8188838B81A0
:10084000898382E066C0CE0160EA70E044E050E057
:1008500064D084E05EC08A819B8190930301809381
:100860000201892B31F481E090E0909303018093A1
:1008700002018091020190910301969587959093D2
:10088000050180930401892B09F042C081E090E0CA
:1008900090930501809304013BC01C81110F8A8154
:1008A00080FD1160898180FD04C081E08BDE81E0E4
:1008B00091DE80E087DE80E08DDE812FADDE882353
:1008C00041F482E080930C0110920E0110920D0110
:1008D00010C081E080930C012E813F8130930E0186
:1008E00020930D01898180930F0181FF03C0232B89
:1008F00009F48BDE8A8180FF0BC08E819F81892B5A
:1009000039F08FEF06C080910C01888381E001C02F
:1009100080E0DF91CF911F910895FB01DC0102C0BF
:1009200005900D9241505040D8F70895DC0101C068
:0E0930006D9341505040E0F70895F894FFCFCA
:06093E00D25A0A00050078
:00000001FF
